:0600000000008A01342813
:08000800FC000308FD000A08DA
:10001000FE00831203137008D8007108D90072081B
:10002000DA007308DB007408DC007508DD00760870
:10003000DE007708DF0089205808F0005908F10039
:100040005A08F2005B08F3005C08F4005D08F50054
:100050005E08F6005F08F7007E088A007D088300CE
:100060007C0809003A3400348330831681008312FF
:100070008B120B17313090006030F800AC20402814
:10008000831203138B168B172208F0002308F1004C
:100090000130F2000030F300B62083120313700821
:1000A000A2007108A3002208F0002308F1006430C8
:1000B000F2000030F300E0200030F2000030F300E6
:1000C0002F2103196628F001F1016A280130F000A0
:1000D0000030F100F201F3012F2103198628831269
:1000E00003132208F0002308F1004A213230F00007
:1000F0000030F1007B21831203132008F000210857
:10010000F1004A210D3075210A3075214428630021
:100110008728831203130B1D92280130F000003052
:10012000F1009428F001F101F201F3012F210319EC
:10013000AB28831203132008F0002108F1000130DE
:10014000F2000030F300B620831203137008A00001
:100150007108A1000B110800673083160313990082
:100160001815981683121816981708007208F007C9
:1001700073080318730AF10708008B13F900780855
:10018000840079088000F80A8B1708008B13F803A5
:100190007808840000088B1708000310F20DF30D97
:1001A000F40BCD2808000310F30CF20CF40BD32849
:1001B00008007208F0027308031C730AF1020800B9
:1001C000F601F701720873040319FF340130F400DB
:1001D00073080038031DF7287208013A031DF72839
:1001E0007008F6007108F700F001F10100347008A2
:1001F0007104031DFC280034F31B0729F40A74085A
:10020000BD200130F400CD20C620F400FC28720887
:10021000BD207308BD207608F2007708F30074084B
:10022000BD200130F400CD20C620F4007208F60095
:100230007308F700C620F300C620F200D920031887
:100240002329B62024297614F403031900347408F2
:10025000BD200130F400D320C620F4000729730824
:100260007102031D0800720870020800003071045A
:10027000031D0800F0040800700FF103F10AF000FC
:1002800071040800F009F1093C29F11F4A292D30B9
:1002900075214221D001D101D201D301D401053011
:1002A000F500F5030A30F200F301E0205030750745
:1002B00084007008303E80007608F0007708F10076
:1002C00036210319672975080038031D51290030AC
:1002D000F4005030740784000008031D7521F40AEF
:1002E0007408053A031D69290800831203130C1EC4
:1002F0007729990008008221003803190800752128
:0C0300003C217B2971088A0070088200F3
:00000001FF
